:10010200120100020000004005168080000001027A
:020112000001EA
:0A0116000A0600020000004001008C
:100122000902270001010080320904000003FF00D8
:10013200000007058102400000070582020002005C
:07014200070588020002001E
:10014A000902270001010080320904000003FF00B0
:10015A0000000705810240000007058202400000F6
:07016A0007058802400000B8
:100172001403000000000000000000000000000066
:10018200000000000C0341004300430045005300FF
:100192001E035700410054004300480044004F0032
:1001A2004700000000000000000000000000000006
:0A31060000010202030304040505A2
:10008000EC4EFEED4F2406F58274313EF583E49389
:10009000FF3395E0FEEF24A1FFEE34E68F82F58377
:1000A0002290E6BCE0547EFF7E00E0D394807C008A
:1000B00022F0E52C2401FFE4352BFEE4352AFDE493
:1000C00035298F2C8E2B8D2AF52922AF30AE2FADFE
:1000D0002EAC2DAB2CAA2BA92AA829C3020819E5FE
:0C00E00036252CF582E535352BF5832202
:10199800E4F534F533F532F531C23CC239C23BC205
:1019A8003A1224A07E017F028E0A8F0B75120175F0
:1019B800131675080175092275100175114A7514F9
:1019C80001751572EE54E07003021A8475350075BE
:1019D80036808E378F38C374B09FFF74019ECF2432
:1019E80002CF3400FEE48F308E2FF52EF52DF52C26
:1019F800F52BF52AF5291200CB500A1200DF74CD19
:101A08001200B180F1E4F52CF52BF52AF529120026
:101A1800CB5017E538252CF582E537352BF583E0D3
:101A2800FF1200DFEF1200B180E485350A85360B1E
:101A380074022480FF740134FFFEC3E5139FF5137D
:101A4800E5129EF512C3E50D9FF50DE50C9EF50C0C
:101A5800C3E50F9FF50FE50E9EF50EC3E5099FF54B
:101A680009E5089EF508C3E5119FF511E5109EF5F7
:101A780010C3E5159FF515E5149EF514D2E843D873
:101A88002090E668E04409F090E65CE0443DF0D23E
:101A9800AFD241122C6790E680E054F7F0538EF8ED
:101AA800C23C303A05121359C23A303C2912316708
:101AB8005024C23C122D6420391690E682E030E7AB
:101AC80004E020E1EF90E682E030E604E020E0E484
:0B1AD800122C96123169121FB880C753
:1013590090E6B9E012087713FD0014510114AB03AC
:10136900137C0613F70813F10913E50A13EB0B00B5
:101379000014E2121EFE40030214EE90E6BBE024C4
:10138900FE602214603324FD60111460222406706B
:1013990048E50A90E6B3F0E50B8037E51290E6B32D
:1013A900F0E513802DE50C90E6B3F0E50D8023E51B
:1013B9000E90E6B3F0E50F801990E6BAE0FF122C23
:1013C900C2AA06A9077B01EA494B600DEE90E6B374
:1013D900F0EF90E6B4F00214EE0214E712312402A1
:1013E90014EE12311A0214EE122E920214EE123178
:1013F900100214EE12316140030214EE90E6B8E0D7
:10140900247F60151460192402703AA239E4332547
:10141900E0FFA23BE4334F8018E490E740F08016E8
:101429001200A140047D0180027D00120080E05479
:101439000190E740F0E4A3F090E68AF090E68B741F
:1014490002F00214EE0214E712316340030214EEB3
:1014590090E6B8E024FE6016240260030214EE90C0
:10146900E6BAE0B40105C2390214EE0214E790E6C7
:10147900BAE0702C1200A140047D0180027D0012A7
:101489000080E054FEF090E6BCE05480131313543E
:101499001FFFE0540F2F90E683F0E04420F08045D1
:1014A900803C123165503E90E6B8E024FE601A2473
:1014B90002703290E6BAE0B40104D239802790E68E
:1014C900BAE0B40202801E80151200A140047D0119
:1014D90080027D0012008080081220ED500790E6FE
:0C14E900A0E04401F090E6A0E04480F098
:0114F50022D4
:0300330002315A3D
:04315A0053D8EF3225
:102DF500E4FFFE7D807C471201B5020401E4FBFA85
:102E0500903F8012082A0202ADE6FE08E6F58BEE39
:032E1500F58D2216
:101E9D008F448E438D428C41E4FFFEFDFCAB44AA82
:0F1EAD0043A942A84174E012034C7003C28E2275
:101EBC00E589540F4410F589538EEF79407841121F
:101ECC002E02AB44AA43A942A8411202AD8F488E00
:101EDC00478D468C45AB48AA47A946A845122DF517
:101EEC00781DA60608A607C28E18122E0ED2ABD2EB
:011EFC008E57
:011EFD0022C2
:0827A0008F448E438D428C41F1
:1027A80079807840122E02AB44AA43A942A841126C
:1027B80002ADAB07AA06A905A804122DF5AD07AC12
:1027C80006E4F5C8438E20AF04ECF5CB8FCDAF05FA
:0B27D800EDF5CA8FCCD2BDD2ADD2CA45
:0127E30022D3
:03001B00022E565C
:102E5600C0E0C0D075D000C000C006781D122E0E8E
:0E2E6600A291B39291D006D000D0D0D0E0322D
:03002B000227E4C5
:1027E400C0E0C0F0C083C082C085C084C086758646
:1027F40000C0D075D000C000C003C004C005C0062E
:10280400C007122CEEC2CFD007D006D005D004D01A
:1028140003D000D0D0D086D084D085D082D083D0CD
:04282400F0D0E032DE
:10238500456E61626C652041444300446973616236
:102395006C65204144430041434345532050434924
:1023A500652D5744472D43534D41204331002D534F
:1023B5003031204D6F646500504349652D574447C2
:1023C5002D43534D4100504349652D5744472D43F7
:1023D500534D00414343455320504349652D5744D0
:0623E500472D3F3F3F00C1
:0F302800C13FC13D0194FFC13E016900016A64CF
:10180F00E6FF7843E475F001120867EF020770E610
:10181F00FFAE3F053F74402EF582E434E7F5832297
:10182F001207707843E475F001020867EE75F00354
:10183F00A42410F582E4343FF5832290E6BDE0FE48
:10184F0090E6BCE02400FDEC3EFC90E6BFE0FE908D
:10185F00E6BEE07A002400FBEA3EFA22E090E74081
:10186F00F0E490E68AF090E68B22E5801313543F64
:10187F00227D017B007A0079807E00020986EE7559
:10188F00F003A42412F582E4343FF58322253AF5C0
:10189F003AE53D3539F539C3E53C953EF53CE53B39
:1018AF00953DF53B227586005391EF90E65D2274CE
:1018BF00402540F58274E7353FF58322C2AFAE3D38
:1018CF00AF3E78807C00FD7B017AE7794022AD3E08
:1018DF007AE779407F40AB072290E6BBE0FE90E6C7
:1018EF00BAE07C002400FFEC3EFE227D017B007AF3
:1018FF000079987E0012098690E74022C3E5409553
:10190F003EE53F953D227C037DE81207A4EF788EDC
:10191F00F6EE08F622E490E68AF090E6BEE090E656
:10192F008BF02275F003A42411F582E4343FF58384
:10193F002290E68AE53EF090E68BE53DF022E53A0F
:10194F002540F582E539353FF5832274002539F9B5
:10195F00EE34FCFA7B0122F582E4343FF5832285D5
:10196F000D82850C83A37402F022850F82850E836E
:10197F00A37407F022D3E53E9400E53D940022D3F3
:09198F00E53E9400E53D940022C0
:0F306D0090E6C2E02041044402F02254FDF0221C
:0F307C0090E6C2E02041044401F02254FEF0220D
:0F308B0090E6C2E02041044404F02254FBF022FE
:0F309A0090E6C2E02040044402F02254FDF022F0
:0F30A90090E6C2E02040044401F02254FEF022E1
:0F30B80090E6C2E02040044404F02254FBF022D2
:07314700EFF490E6C2F02254
:03315E00D29522E5
:1000EC00D295E4FFFE000FBF00010EBE04F7BFB0B7
:0300FC00F4C295B6
:0100FF0022DE
:06286B008B428A43894400
:102871008B458A4689477845121834E5231207703B
:1028810090E685E0FF7845121834EF12077090E664
:1028910084E0FF7845121834EF120770784512185A
:0B28A10034ED120770C3E5479544FFBB
:0128AC002209
:062295008B408A418942E2
:10229B008B438A448945121832E52312182FE52205
:1022AB0012182FE52112182FE52512077078A612A8
:1022BB00180F78A512180F787E12180F787D121848
:1022CB000F787412180F787312180F787612180F84
:1022DB00787512180F787812180F787712180F7804
:1022EB007A12180F787912180F121832E524120788
:1022FB0070787F12180F789312180F789512180FA9
:10230B00787B12180F787C12180FC3E5459542FFA6
:01231B00229F
:0528AD00E5AA30E63A47
:1028B2007539017E0012195A78A4E6FD12286BEFD1
:1028C2002539F539E478A4F612195A122295EF2522
:1028D20039F539E4787FF6F52490FC00E539F0907B
:0A28E200E69C7402F0E490E69DF01D
:0128EC0022C9
:07314E00EF448078A4F62293
:072C3800AD07E5AA30E0271B
:102C3F007541017E0074002541F9EE34F0FA7B01F5
:102C4F0012286BEF2541F54190F000F090E690745B
:072C5F0002F0E490E691F0A1
:012C6600224B
:102FEF00200710D207D23EC2007F01122C387F0576
:042FFF00121DDD22A0
:102ECE00203D19D23DD2947890E6FBF460077D0147
:0D2EDE007F0B122F58D2077F06121DDD2238
:102A5C00EF30E505903F02EDF0EF30E405903F03D9
:102A6C00EDF0EF30E305903F09EDF0EF30E205902B
:102A7C003F08EDF0EF30E105903F07EDF0EF30E06F
:072A8C0005903F06EDF0226A
:1026C8008F41E541C3941F500280027F1F8F41E56F
:1026D80041C3941F501778407CE77F0E121880780A
:1026E8004D7CE77F0A1218FA7418F0801578417C3F
:1026F800E77F1212188078537CE77F0C1218FA745F
:092708001FF0121870E541F022E7
:1014F6008E398F3A8C3B8D3C8A3D8B3E90E6B8E028
:1015060030E70302167A123016121984404D12196A
:101516002490E6A0E020E1F9E53E6412453D70081E
:101526001218CB1209868029E53E640E453D6003FC
:0315360002168416
:101539001218CB120986788176027884E6FE18E6BD
:10154900FDEEF53FEDF540FF1219150876FFD2AF14
:061559007882E6FF7E002F
:10155F00805BE53C853BF012089D15D3000115F526
:10156F00000215B8004415BF004515A8004915AD78
:10157F00004A15A5005215C5005415CC005515B2DB
:10158F00006915B5006A15F88000161680011666F9
:10159F0080020000168402305CE4FF022C387F02C8
:1015AF0002314E022F9B022FB0AF3AAE39022D16E9
:1015BF00E53A7890F622AF3AAE3902303AAF3AAE0A
:1015CF0039022E74308703021684E539453A24FF19
:1015DF00B39295E53A453970047F0180027F00EFA1
:1015EF0024FFB3923F22022545E4FBFD7F08122F13
:1015FF00587F007E007D007C00121E9D308705C243
:10160F0090C29122C29122308733E539700EC29178
:10161F00FBFD7F08122F58C291C29022E539FFBF00
:10162F000105308613800CEF64027049E53AC394CC
:10163F00805005C290D29122C291D29022E539FFFB
:10164F00BFFF09E53AFB7DFF7F08801CAC39AD3A3F
:10165F00E41203C8021E9DC3E539948040047F093C
:10166F0080027F0A7B507D02022F58121984400599
:06167F00AF3E1226C82256
:101CEC008F398D3A8B3B90E6B8E030E703021D80CC
:101CFC00E53D7074E53E7070E53C7F00FEEF253BE2
:101D0C00FFE43EFEEF8EF012089D1D5200001D57A1
:101D1C0000011D6101001D6101011D6101021D61B8
:101D2C0001031D6101041D6101051D6101061D6199
:101D3C0001071D6101081D6101091D61010A1D6A70
:101D4C00FFFF00001DDCAF39022A93E539FD7C0052
:101D5C00AF3A02217BAB39AD3AAF3B022F58E53A93
:101D6C00606EAD39FF022A5C12194090E6A0E0309B
:0B1D7C00E15E80F7E53DD39400405588
:101D8700753F017440253FF9E434E7FA7B017DFF95
:101D970012286BEF253FF53F2440F9E434E7FA7B3F
:101DA70001122295EF253FF53FE4787FF6F524E50C
:101DB7003BB4010C12292DAE3F053F121824EFF05A
:101DC70090E740E53FF0121940E53A7008E539B46D
:051DD70001031230D5EC
:011DDC0022E4
:1020ED0090E6B9E012087721161021161121334020
:1020FD002172A22172A32146D42159D52160D62166
:10210D0065D7216DD80000217790E6BAE0FFA3E0F6
:10211D00FDA3E0FBA3E0F53CA3E0F53DA3E0F53E18
:10212D00121CEC0221791218E8C006C00712184AD9
:10213D00D007D0061214F680331218E8C006C00777
:10214D0012184AD007D006120EF080207F01122CF3
:10215D003880081228AD8003122632123016800CFA
:0E216D00122D648007121BEB8002D322C322C6
:100EF0008E398F3A8C3B8D3C8A3D8B3E90E6B8E034
:100F000030E7030210B012198E400A12192490E63D
:100F1000A0E020E1F9E53A8539F012089D0F9D0027
:100F200001101300A00FDE00B00FA900D010420185
:100F3000A0103C01A1103601A2103001A3102A011B
:100F4000A4102401A5101E01A6101801A7100D0160
:100F5000B0100701B1100101B20FFB01B30FF50191
:100F6000B40FEF01B50FE901B60FE301B70FD801D8
:100F7000D00FD201D10FCC01D20FC601D30FC001C7
:100F8000D40FBA01D50FB401D60FAE01D71048FF68
:100F9000001080FF0110A2FF0200001358E53C542E
:100FA0000175F011A490E6C2F0E53CF5B022E53CF5
:100FB0001392B722E53C1392B622E53C1392B52278
:100FC000E53C1392B422E53C1392B322E53C139224
:100FD000B222E53C1392B122E53C1392B022E53CEB
:100FE000F59022E53C13929722E53C13929622E578
:100FF0003C13929522E53C13929422E53C13929384
:1010000022E53C13929222E53C13929122E53C1397
:10101000929022E53CF58022E53C13928722E53C44
:1010200013928622E53C13928522E53C139284229A
:10103000E53C13928322E53C13928222E53C139215
:101040008122E53C1392802212198E50030213581C
:10105000AE3DAF3E7C007D031207B6ED4C6003024F
:101060001358D3E53E9430E53D94004003021358F5
:10107000AE3DAF3E78107C3F7D011218D602098646
:10108000AF3CE53CBF010D1200ECD23F7BFF7A2361
:101090007985800B12315EC23F7BFF7A2379900203
:1010A00028EDAF3CBF0103D38001C392410231550B
:1010B000E53A8539F012089D13320002134B000304
:1010C000124800A011C000B0113800D012C001A019
:1010D00012B001A112A001A2129001A3128001A4DA
:1010E000127001A5126001A6125001A7123801B0BA
:1010F000122801B1121801B2120801B311F801B49B
:1011000011E801B511D801B611C801B711B001D06D
:1011100011A001D1119001D2118001D3117001D41D
:10112000116001D5115001D6114001D712D0FF0036
:1011300012E6FF010000135890E740E5B00213519A
:1011400030B7047F0180027F0090E740EF02135127
:1011500030B6047F0180027F0090E740EF02135118
:1011600030B5047F0180027F0090E740EF02135109
:1011700030B4047F0180027F0090E740EF021351FA
:1011800030B3047F0180027F0090E740EF021351EB
:1011900030B2047F0180027F0090E740EF021351DC
:1011A00030B1047F0180027F0090E740EF021351CD
:1011B00030B0047F0180027F0090E740EF021351BE
:1011C00090E740E5900213513097047F0180027F41
:1011D0000090E740EF0213513096047F0180027FB8
:1011E0000090E740EF0213513095047F0180027FA9
:1011F0000090E740EF0213513094047F0180027F9A
:101200000090E740EF0213513093047F0180027F8A
:101210000090E740EF0213513092047F0180027F7B
:101220000090E740EF0213513091047F0180027F6C
:101230000090E740EF0213513090047F0180027F5D
:101240000090E740EF02135190E740E58002135110
:101250003087047F0180027F0090E740EF02135146
:101260003086047F0180027F0090E740EF02135137
:101270003085047F0180027F0090E740EF02135128
:101280003084047F0180027F0090E740EF02135119
:101290003083047F0180027F0090E740EF0213510A
:1012A0003082047F0180027F0090E740EF021351FB
:1012B0003081047F0180027F0090E740EF021351EC
:1012C0003080047F0180027F0090E740EF021351DD
:1012D000AE3DAF3E78407CE77D017B017A3F7910DF
:0612E0001209860213440E
:1012E600E4F53F78A9E6FE08E6FDAC3F053F74400D
:1012F6002C121827EDF0EE12181FEFF0789F121837
:101306001EEFF00812181EEFF0121820E56DF0E53A
:101316006C12181FEFF0D3E53F953EE4953D40046F
:0C132600AF3F8002AF3E90E68BEFF0225C
:1013320090E6F4E020E1047F0180027F0090E74024
:10134200EFF090E68BE53EF02212187990E740F03C
:0713520090E68B7401F0220C
:10301600C2AFE4F56CF56DD2AFC23DD2007F0402BB
:023026001DDDAE
:0D30E300C2AF056DE56D7002056CD2AF2225
:102E7400AB07AA06C2AF7C037DE81207B6EF7883DE
:0E2E8400F6EE08F6EB788EF6EA08F6D2AF22EC
:10303A00AA06C2AFEF7883F6EA08F6121915D2AFDC
:01304A002263
:10168500AF23E5805403C454F0FEE5B0540F4EF586
:1016950023E5236F787F46F6A21B301301B350254F
:1016A500903F0FE014F0E07024A21B301301B372D9
:1016B500239223A21B9213A213720B920BA22BA0AF
:1016C50013922B8000903F09E0903F0FF0A21A3053
:1016D5001201B35025903F0EE014F0E07024A21AD9
:1016E500301201B372229222A21A9212A212720A27
:1016F500920AA22AA012922A8000903F08E0903F09
:101705000EF0A219301101B35025903F0DE014F0F1
:10171500E07024A219301101B372219221A219920D
:1017250011A21172099209A229A011922980009093
:101735003F07E0903F0DF0A218301001B3502590FF
:101745003F0CE014F0E07024A218301001B37220B1
:101755009220A2189210A21072089208A228A01036
:1017650092288000903F06E0903F0CF0A21D3015B6
:1017750001B35025903F05E014F0E07024A21D3020
:101785001501B372259225A21D9215A215720D920F
:101795000DA22DA015922D8000903F03E0903F05EE
:1017A500F0A21C301401B35025903F04E014F0E082
:1017B5007024A21C301401B372249224A21C92142A
:1017C500A214720C920CA22CA014922C8000903FB3
:1017D50002E0903F04F07893E6552455227895462B
:1017E500F6787BE65524FFE522F45F0846F6789205
:1017F500E6F4552460057F0212314E787FE66005D8
:091805007F0212314E7892A624F4
:01180E0022B7
:10217B00EF12087721A40021AC0121B40221BC038A
:10218B0021C40421FA0521EF0621E40721CC082103
:10219B00D40921DC0A00002205EC4D24FF92B78004
:1021AB005BEC4D24FF92B58053EC4D24FF92B6802F
:1021BB004BEC4D24FF92978043EC4D24FF9296807D
:1021CB003BEC4D24FF92918033EC4D24FF92938096
:1021DB002BEC4D24FF92928023EC4D24FF92411265
:1021EB00306D8018EC4D24FF924112307C800DEC49
:0E21FB004D24FF924112308B8002C322D3226A
:10205400EF12087720800020880120900220980346
:1020640020A00420D60520CB0620C00720A80820E5
:10207400B00920B80A20E10B000020E9EC4D24FF50
:1020840092B78063EC4D24FF92B5805BEC4D24FF46
:1020940092B68053EC4D24FF9297804BEC4D24FF75
:1020A40092968043EC4D24FF9291803BEC4D24FFAB
:1020B40092938033EC4D24FF9292802BEC4D24FFBD
:1020C400924012309A8020EC4D24FF92401230A9A5
:1020D4008015EC4D24FF92401230B8800AEC4D2458
:0920E400FF92948002C322D32272
:102A9300903F10E07005EFA2E392B7903F13E07010
:102AA30005EFA2E192B5903F16E07005EFA2E29226
:102AB300B6903F19E07004EF139297903F1CE070BB
:072AC30005EFA2E492962248
:10292D00E4FF3097047E0180027E00EE420730B551
:10293D00047E0280027E00EE420730B6047E0480E3
:10294D00027E00EE420730B7047E0880027E00EE64
:0E295D0042073096047E1080027E00EE420794
:01296B002249
:1023EB00EF14601914601F14602914603314603DDE
:1023FB00240570497FE312313778A5803B7FE512C6
:10240B003137787D8032C293C2927FEE12313778AA
:10241B00738025C293D2927FEE1231377875801874
:10242B00D293C2927FEE1231377877800BD293D250
:0E243B00927FEE1231377879A60608A60722A6
:10304B00AF6905691223EBE56975F0068485F069B4
:01305B002252
:102F8600E4F541E4FBFDAF41122F580541E541C38D
:042F9600941040EF64
:012F9A002214
:102F5800AE07C2AF12188DEFF0121932EBF0EF1274
:062F6800183CEDF0D2AFB1
:012F6E002240
:10271100E4FE78940612183BE0D394004034789498
:10272100E6FB700E12188DE0FF7D017C0012205433
:102731008020EE121932E06B701812188DE0FFE460
:10274100FDFC12205412183BE0F4600612183BE025
:0827510014F00EEE641070BDDF
:01275900225D
:0E30C700E4F5B275B3FF75B5F090E6C3F022E4
:10296C007898760C087602087601E408F630B10403
:10297C007F0180027F00EF25E025E04463FF30B04B
:10298C00047E0180027E00EE25E04FF520789CF657
:0F299C00E408F608F678A3F6C294C207C29122A7
:1026320090E61274E0F000000090E615F000000051
:1026420090E611F000000090E610E0547FF00000E8
:102652000090E613E0547FF000000090E614E0548E
:102662007FF0000000122F9B122FB090E6837412AD
:0C267200F07432F090E65CE04402F022CC
:0E30D500E4F521F525F5247895F6787CF622B1
:102BD300903F027401F0903F04F0903F03F0903F68
:102BE30005F0903F09F0903F0FF0903F08F0903FC1
:102BF3000EF0903F07F0903F0DF0903F06F0903FAE
:032C03000CF022B0
:1025E5007F07123147E478A7F608F6D200C23EC24B
:1025F5003DC207C2977880761208760208F608F67B
:1026050008F6788EF608F60876FF7885760108F6DE
:1026150008F63087047FFF80027F007888A60708C8
:0D2625007601087601E408F608F608F622B2
:1024A0007F01121DDD12315E12313F903F017451E8
:1024B000F0903F0B7401F090E600E054E74410F018
:1024C000903F801208364C371B00122ACA122A236A
:1024D00012263212254543AF017BFF7A23799C12E5
:1024E00028ED3087097BFF7A2379B31228ED7F022C
:0324F000021DDDED
:101FB800303F0F78AAE6656B600812304B78AAE6C6
:101FC800F56BD37997E778AA9619E718965005C262
:101FD8004112306D7882E66034203E17788FE6FE35
:101FE80018E6FDEDFFD3E56D9FE56C9E401F122FAF
:101FF800EF801A788FE6FE18E6FDEEFCE56CC31359
:10200800FEE56D13D39DEE9C4003122ECEA2809266
:1020180002A2B09203789CA620AE6CAF6D7C037DC3
:10202800E81207B6EF789FF6EE08F6E56D08F6E5D4
:102038006C08F678A4E6C3948040031228AD308774
:0C2048000A90E6F4E020E003122ECE2205
:102F9B0090E6047480F00000007402F0000000E47E
:052FAB00F0000000220F
:102FB00090E6047480F00000007408F0000000E463
:052FC000F000000022FA
:10305C007F007E007D007C00121E9D1225E502295A
:01306C006CF7
:10254500E478A4F67F07123147122FB0122F9B783B
:1025550093763F787B763FE47892F6C23DC2B7C268
:1025650094C207C2911230D5122BD3122F867F0049
:102575007E007D7A7C441227A01230C712305C3071
:1025850087097B507D027F0A122F587F0102314750
:102ACA00E4F5391218DF7D087FF87E1D122595E49A
:102ADA00F53974402539121827E0FDE53975F002F9
:102AEA00A42474F9740135F08982F583EDF005396F
:052AFA00E539B408DD20
:012AFF0022B4
:062449008B398A3A893B41
:10244F00E4F53C122FDA8F3DE53D25E024029001A3
:10245F0092F0E4F53CAF3DEF3395E0FEC3E53C9FD2
:10246F00EE6480F87480985027AB39AA3AA93B855F
:10247F003C82758300120743FDE53C75F002A424EE
:10248F0094F9740135F08982F583EDF0053C80C530
:01249F00221A
:102A23001218DF7D017F037E0012259590E740E0B9
:102A330090010CF090E740E0247F600B0470107B62
:102A4300FF7A2379BD800E7BFF7A2379CB80067BC7
:092A5300FF7A2379D812244922EC
:09312E00788276017F03021DDDA9
:102D1600EF4E60047F0180027F007882EFF6600448
:102D26007F0380027F07121DDD7882E67008121885
:072D36007970031230F02256
:102CEE001227111216851230E3D56A1B78AA06E652
:102CFE0018700106C378AAE6940A18E694004004F8
:072D0E00E4F608F6756A64A3
:012D1500229B
:102FC5007B807DFF7F03122F58D297C24112307C40
:052FD500C24102308B37
:0B30F000C2977B80E4FD7F03022F5895
:101DDD00EF1208771DFA011E17021E25031E32048D
:101DED001E5A051E6B061E8D0700001E9C7FFF12DE
:101DFD002A93E490E6C2F01218797005D2410230B0
:101E0D007C208503021E9C021E9512187970030218
:101E1D001E9C30857A021E951218797003022FC50B
:101E2D0030856C803512187970028003308560D250
:101E3D004112306D78AAE62402FF18E436FE7C00CC
:101E4D007D0A1207B67896A60408A60522121879FF
:101E5D0070057F050231473085357F018017788801
:101E6D00E6600B7F007E007DFA7C44121E9D1218E9
:101E7D007970087F04123147D2B72230851180085E
:101E8D00121879600A3085077F04123147C2B722D4
:102D8900C0E0C083C082C085C084C086758600D279
:102D99003A1218B77401F0D086D084D085D082D089
:042DA90083D0E032C1
:102E1800C0E0C083C082C085C084C0861218B47464
:0F2E280004F0D086D084D085D082D083D0E03221
:102E3700C0E0C083C082C085C084C0861218B47445
:0F2E470002F0D086D084D085D082D083D0E03204
:102B6B00C0E0C083C082C085C084C08675860085E6
:102B7B00100C85110D12196E85080E85090F12198F
:102B8B00791218B77410F0D086D084D085D082D04B
:042B9B0083D0E032D1
:102DAD00C0E0C083C082C085C084C086758600D255
:102DBD003C1218B77408F0D086D084D085D082D05C
:042DCD0083D0E0329D
:1029E800C0E0C083C082C085C084C0867586009060
:1029F800E680E030E71285080C85090D12196E850E
:102A0800100E85110F1219791218B77420F0D0869C
:0B2A1800D084D085D082D083D0E03283
:01316B003231
:01316C003230
:01316D00322F
:01316E00322E
:01316F00322D
:01317000322C
:01317100322B
:01317200322A
:013173003229
:013174003228
:013175003227
:013176003226
:013177003225
:013178003224
:013179003223
:01317A003222
:01317B003221
:01317C003220
:01317D00321F
:01317E00321E
:01317F00321D
:01318000321C
:01318100321B
:01318200321A
:013183003219
:013184003218
:013185003217
:013186003216
:013187003215
:013188003214
:013189003213
:01318A003212
:01318B003211
:01318C003210
:01318D00320F
:01318E00320E
:06282800AB07AA06AC0597
:10282E00E4FD903F0BE0600B7E000DEE2487121945
:10283E0066EAF0AE050D74872E121966EBF0AF0541
:10284E000D74872F121966ECF0903F01E0FF7A3F6E
:0D285E007B87122F07903F01E0FF022B0047
:0A2B36008E418F428D438A448B4587
:102B4000E4F546E546C3954350200542E542AE41D3
:102B50007002054114FFE5452546F582E43544F54C
:0A2B600083E0FD122828054680D905
:012B6A002248
:0A2595008E418F428D438A448B452E
:10259F00E4FDF546903F0BE06012E541FF7E000D34
:1025AF00EE2487F582E4343FF583EFF0AE050D742A
:1025BF00872EF582E4343FF583E542F0903F01E04A
:1025CF00FF7A3F7B87122F07903F01E0FFAB45AAB1
:0625DF0044AD43022EEBA7
:021EFE00D322ED
:102E920000000090E6247402F0000000E490E625B1
:0E2EA200F000000090E6BAE0903F0AF0D32264
:0A311000903F0A12186B04F0D3225E
:0A311A0090E6BAE0903F00F0D322E7
:0A312400903F0012186B04F0D32254
:02316100D32277
:02316300D32275
:02316500D32273
:02316700D32271
:02316900D3226F
:101BEB0090E6BAE0753900F53AA3E0FEEE42399083
:101BFB00E6BEE0753B00F53CA3E0FEEE423B90E613
:101C0B00B8E064C06003021C92E53C453B700302E4
:101C1B001CEB90E6A0E020E1F9C3E53C9440E53BEA
:101C2B0094005008853B3D853C3E8006753D007514
:101C3B003E4090E6B9E0B4A31EE4F53FF54012191F
:101C4B000B503812194DE0FF1218BEEFF00540E5AE
:101C5B004070EB053F80E7E4F53FF54012190B5060
:101C6B00101218BE74CDF00540E54070EF053F80B3
:101C7B00EB1218DDAF3AAE39122595121870E53E0E
:101C8B00F012189C021C1490E6B8E064407051E509
:101C9B003C453B604B121870F090E6A0E020E1F958
:101CAB0090E68BE0753D00F53E90E6B9E0B4A31EDF
:101CBB00E4F53FF54012190B501E1218BEE0FF124F
:101CCB00194DEFF00540E54070EB053F80E712182A
:101CDB00DDAF3AAE39122B36E53E12189C021C9A38
:011CEB0022D6
:03004300021F0099
:03005300021F0089
:101F0000022D8900022E3700022E1800022DAD008E
:101F1000022B6B000229E80002316B0002316C00D9
:101F200002316D0002316E0002316F00023170002B
:101F3000023171000231720002317300023174000B
:101F40000231750002316C000231760002317700F7
:101F5000023178000231790002317A0002317B00CF
:101F600002317C0002316C0002316C0002316C00E5
:101F700002317D0002317E0002317F00023180009B
:101F8000023181000231820002318300023184007B
:101F9000023185000231860002318700023188005B
:101FA0000231890002318A0002318B0002318C003B
:081FB00002318D0002318E00A8
:022DD1008F1C55
:102DD300903F86EDF07A3F7B867D01122F077A3F85
:102DE3007B847D02AF1C122EEB903F84E0FEA3E0B8
:012DF300FFE0
:012DF40022BC
:1029AB00AE07C2E990E678E04480F0EE25E090E6D1
:1029BB0079F090E678E030E0F9ED90E679F090E68A
:1029CB0078E030E0F990E678E04440F090E678E08B
:0D29DB0030E0F990E678E020E6F9D2E9223C
:022F6F00AC07AD
:102F71001229AB7A3F7B877D02122EEB903F87E0CF
:042F8100FEA3E0FFCC
:012F85002229
:08313700AD077F40122F6F224B
:102C960090E682E030E004E020E60B90E682E03049
:102CA600E119E030E71590E680E04401F07F147EFC
:0C2CB6000012275A90E680E054FEF02245
:102D640090E682E044C0F090E681F04387010000E1
:042D74000000002239
:102C670030410990E680E0440AF0800790E680E072
:102C77004408F07FDC7E0512275A90E65D74FFF06A
:0F2C870090E65FF05391EF90E680E054F7F02273
:08313F00E4F51BD2E9D2AF2236
:102B000090E678E020E6F9C2E990E678E04480F0CB
:102B1000EF25E090E679F090E678E030E0F990E695
:102B200078E04440F090E678E020E6F990E678E03E
:062B300030E1D6D2E922DB
:102C0600A90790E678E020E6F9E51B702390E678C0
:102C1600E04480F0E925E090E679F08D16AF03A94F
:102C2600077517018A188919E4F51A751B01D3224D
:022C3600C322B7
:102B9F00A90790E678E020E6F9E51B702590E67826
:102BAF00E04480F0E925E0440190E679F08D16AF1E
:102BBF0003A9077517018A188919E4F51A751B03FC
:042BCF00D322C32228
:03004B00021AE3B3
:101AE300C0E0C083C082C085C084C086758600C044
:101AF300D075D000C000C001C002C003C006C0073B
:101B030090E678E030E206751B06021BCD90E6787E
:101B1300E020E10CE51B64026006751B07021BCD88
:101B2300E51B24FE605F14603624FE7003021BBEB7
:101B330024FC7003021BCA24086003021BCDAB17ED
:101B4300AA18A919AF1A051A8F82758300120743C1
:101B530090E679F0E51A65167070751B05806B9039
:101B6300E679E0AB17AA18A919AE1A8E827583001D
:101B7300120782751B02E5166401704E90E678E049
:101B83004420F08045E51624FEB51A0790E678E078
:101B93004420F0E51614B51A0A90E678E04440F0C4
:101BA300751B0090E679E0AB17AA18A919AE1A8E37
:101BB30082758300120782051A800F90E678E0444D
:101BC30040F0751B008003751B005391DFD007D0D5
:101BD30006D003D002D001D000D0D0D086D084D09C
:081BE30085D082D083D0E032EE
:022CC200A90760
:102CC400AE14AF158F828E83A3E064037017AD0139
:102CD40019ED7001228F828E83E07C002FFDEC3E83
:092CE400FEAF0580DF7E007F00D9
:012CED0022C4
:102EEB00122B9FE51B24FA600E146006240770F367
:0C2EFB00D322E4F51BD322E4F51BD32204
:102F0700122C06E51B24FA600E146006240770F3E2
:0C2F1700D322E4F51BD322E4F51BD322E7
:10275A008E398F3A90E600E054187012E53A240157
:10276A00FFE43539C313F539EF13F53A801590E6CE
:10277A0000E05418FFBF100BE53A25E0F53AE539B9
:10278A0033F539E53A153AAE39700215394E600516
:06279A00122D7880EE22F2
:102D78007400F58690FDA57C05A3E582458370F96E
:012D88002228
:0B30FB002530326258002530345800A8
:02303700C14294
:102F3F00743FF59A7440F59B74E7F59D74C0F59E48
:092F4F00E4227B017A3F79402263
:05315500A2419242229C
:10267E00204204E4FEFF2290E6A2E020E1F9122FB0
:10268E0051122FDAEF2401F544E43EF543122F3FA9
:10269E00FFFEC3EF9544E5436480F8EE64809850E6
:1026AE000F90E67BE090E67CF00FBF00010E80E21B
:0926BE00E54490E68FF0AE43FF05
:0126C70022F0
:1028ED008B408A418942204204E4FEFF22122923B3
:1028FD008E498F4A854046854147854248122F5162
:10290D001224F312292374402FF582743F3EF58370
:10291D00E4F012267E22AB40AA41A942122FDA2200
:10300300204204E4FEFF22903F40EFF0E4A3F012DD
:03301300267E22F4
:102F2300204204E4FEFF227550FF7551307552FBB9
:0C2F33008F53122F51120ADD12267E224D
:102EB000204204E4FEFF227550FF75513175520126
:0E2EC0008E538F54122F51120ADD12267E22DD
:10231C0090E685E02405F56E204204E4FEFF227869
:10232C00407C3F7D01120A6490E6A2E030E1079008
:06233C00E685E0B56EF23B
:10234200122F51122FDAEF2401F572E43EF57112C9
:102352002F3FF56FF570C3E5709572E5716480F8F3
:10236200E56F648098501290E67BE090E67CF00581
:1023720070E57070E1056F80DDE57290E68FF0AE7A
:0223820071FFE9
:012384002236
:1001B20002046DE86480F8E933E83360110460F00A
:1001C200ED33EC337009E8FCE9FDEAFEEBFF2204B3
:1001D20060DED3EB9FEA9EE99DE8C2E78CF0C2F7AE
:1001E20095F0400CE8CCF8E9CDF9EACEFAEBCFFB7A
:1001F20012043885D0F05804700320D5B3E8047097
:10020200075002B2D502047792D5EC0460F7E4CC31
:10021200C0E0C398F8603B94186008400DD0E0FB42
:1002220002044FE4FBFAC9FC8028E830E406E4C982
:10023200FBE4CAFCE830E305E4C9CACBFCE8540796
:100242006010F8C3E913F9EA13FAEB13FBEC13FCA1
:10025200D8F130F52FC3E49CFCEF9BFFEE9AFEED44
:1002620099FDD0E0FBEF4E4D4C701222DB030204ED
:1002720074EC2CFCEF33FFEE33FEED33FDED30E793
:10028200EB02044FEF2BFFEE3AFEED39FDD0E0FB1F
:1002920050130BBB0003020477ED13FDEE13FEEFC8
:0802A20013FFEC13FC02044FF2
:1002AA00020477EC5D046005E85904700302046DEA
:1002BA00120438580460F6EC4860F2EC7004FDFE53
:1002CA00FF22C860DB2481C85009C3986002500627
:1002DA000204749850CAF582E9294B4A7005AB8228
:1002EA0002046375F0007C1A7880C3EF9BEE9AEDE6
:1002FA0099400DC3EF9BFFEE9AFEED99FDE842F09F
:10030A00DC23ACF0D0E0FFD0E0FED0E0FDAB8220F1
:10031A00E7101BEB60BAEC2CFCEF33FFEE33FEED7B
:10032A0033FD02044FE803F830E705C0F075F0002A
:10033A00EF2FFFEE33FEED33FD40B830E7C280AA5F
:10034A0074F8CC6480CCC86480C8F58204604FC35A
:10035A00EB9FF5F0EA9E42F0E99D42F0E89C45F0F9
:10036A00603C501DE5825FFFE582D313CB5BCBF483
:10037A002B5582FB50280ABA002409B900200880AC
:10038A001DE5825BFBE582D313CF5FCFF4C3132F46
:10039A005582FF50090EBE00050DBD00010CC3EBCE
:1003AA009FF5F0EA9E42F0E99D42F0E89C45F06034
:0903BA0007CC4820E701B3EC2256
:1003C30075F020800E75F010800575F0087D007EB5
:1003D300007F003392D530D50312080BEC33401065
:1003E300EF33FFEE33FEED33FDEC33FCD5F0ED22BE
:0E03F300E5F0247EA2D513CC92E7CDCEFF22FA
:10040100EDD2E7CD33EC3392D524814006E4FFFEF3
:10041100FDFC22FCE4CFCECDCC24E0501174FF8052
:10042100EDC3CC13CCCD13CDCE13CECF13CF0470EF
:07043100F030D5DE02080BDC
:100A8100E5642450F8E6056422784D303702785049
:100A9100E475F00112086702072A2030EB7F2ED29D
:100AA100308018EF540F2490D43440D4FF30340BED
:100AB100EF24BFB41A0050032461FFE565600215FD
:100AC100650568E5687002056730370D784DE47596
:100AD100F001120867EF020770022D3D7403D2374F
:100AE1008003E4C237F5648B4D8A4E894FE4F56586
:100AF100F567F568E56560077F20120ABC80F5752A
:100B010066FFC231C230C232C233C235C236C238C8
:100B1100120A8AFF700D3037057F00120ACDAF68C7
:100B2100AE6722B4255FC2D5C234120A8AFF24D02F
:100B3100B40A00501A75F00A786530D50508B6FF79
:100B41000106C6A426F620D5047002D23380D9242A
:100B5100CFB41A00EF5004C2E5D234020DBAD2313B
:100B610080C6D23080C0D23280BCD2D580BAD235D4
:100B710080B47F20120ABC2032077401B5650040A1
:100B8100F1120A81FF120ABC020AF5D238D236806C
:100B910095120A81FB120A81FA120A81F94A4B70F5
:100BA1000679B17A0E7BFF20322EE565602A7E0040
:100BB1008E8275830012074360060EEE656670F043
:100BC100C2D5EBC0E0EAC0E0E9C0E0EE120E1AD0F7
:100BD100E0F9D0E0FAD0E0FB12072AFF60AAEBC0EF
:100BE100E0EAC0E0E9C0E0120ABCD0E02401F9D09B
:100BF100E03400FAD0E0FBE5660460DCD566D9801C
:100C010087D23280A2120DFD60F7E56670010412F1
:100C11000482A966600DE566600914F566120EA4EA
:100C2100EF60F3EA30E702F404C3995077EAF42560
:100C3100660430E701E404F566800D120DFD60C124
:100C4100EA05662566120482EA7863F630E701E474
:100C5100256604D5660420350114120E1AE4C0E09D
:100C6100120EA47863E6601320E70714F6120AA4B3
:100C7100802204F6D0E014C0E07F00120AA4E566E9
:100C81006007120A9B1566800B303503120A9BD050
:100C9100E0020AF5D0E00480C5120DFD60A0E56612
:100CA100041204827863EAF6E566203502600104E5
:050CB1002404120E1ADC
:100CB60074FF04C0E0120EA4120AA4E566203502F1
:100CC6006003120A9BD0E0B566E87F45120AAE784B
:100CD60063E67F2B30E7047F2DF404C0E0120ABCE4
:100CE600D0E075F00A84C0F0120AA5D0E0120AA579
:100CF600020AF5791080027908C236C2388008D215
:100D0600D5790A8004790AC2D5E566047002F566CB
:100D1600E4FAFDFEFF120A81FC7B08203113120A59
:100D260081FD7B1030300A120A81FE120A81FF7B98
:100D360020EC3382D592D55013C3E43030069FFFA2
:100D4600E49EFEE42031039DFDE49CFCE4CBF8C266
:100D560031EC700CCFCECDCCE824F8F870F38017C8
:100D6600C3EF33FFEE33FEED33FDEC33FCEB33FB29
:100D7600994002FB0FD8E9EB303105F8D0E0C448C2
:100D8600B231C0E00AEC4D4E4F78207B0070C2EACB
:100D9600B5660040BCC0E0120E1CD0F0D0E0203199
:100DA60004C4C0E0C4B231C0F0120AA5D0F0D5F038
:100DB600EB020AF51208770B92530CF9580B634CA9
:100DC6000B5F420CFD4F0D05440D05490B78430D95
:100DD6000B550C3C460C9A450C06470ED1500B673A
:100DE6002D0B6B2E0B8E2B0B6F230B8C200EBA2A22
:100DF6000B274800000B86E566B4FF0375660612EE
:100E06000A81FC120A81FD120A81FE120A81FF780C
:100E16005C0204B1790AA2D5203314303509B91021
:100E2600020404B9080104A2D520360250010420A8
:100E360032689232B565005034C0E07F20303319F5
:100E46007F30A23272367235500F120E73C232C222
:100E560036C235C2387F30800F303503E9C0E01224
:100E66000ABC303503D0E0F9D0E0B565CC30351793
:100E76007F30B9100C120ABC7F583034077F788057
:100E860003B90803120ABC3032057F2D020ABC7F63
:100E9600202038F87F2B2036F322923280CF7F0035
:100EA600B407005005245CF8E6FF22286E756C6CCA
:100EB6002900D231120A813031F8C231786530D535
:100EC6000108F6020B272D50434958120A812403C4
:100ED600B405004001E4900ECC93120AAD743A12A8
:0A0EE6000AADD233756504020CF961
:10043800E9D2E7C933E833F892D5EDD2E7CD33EC0A
:0704480033FC5002B2D52283
:10044F00EC30E7100FBF000C0EBE00080DBD00040E
:10045F000BEB6014A2D5EB13FCED92E7FD2274FFBA
:10046F00FCFDFEFF22E480F8A2D574FF13FC7D8013
:03047F00E480EF27
:10048200F920E72824F950037907E4F42402FB1841
:10049200DBFDE624FB5014E9600DE4F618E604F6F1
:0F04A200B40A08E4F6D9F57401F60A22C2D5228D
:1004B100ED33EC3392D5FA602AB4FF33EDC2E77B1A
:1004C100FF60067A0479D6E4227A0479DF20D50424
:1004D1007A0479DA224E614E002B494E46002D49AD
:1004E1004E4600E47A08F608DAFC7B00740722E83D
:1004F100C0E0ECC0E0EDC0E0EEC0E0EFC0E0EA75C6
:10050100F010A4CAABF075F04DA42BFBE435F0FC60
:10051100EA2410FAEB34C5FBEC34D9FCEDC2E7FF59
:1005210075F056A4F42411C5F0F434C58FF0A42A53
:10053100E5F03BE43CF620E7141206EAD0E0FFD0F8
:10054100E0FED0E0FDD0E0FC1202AD8014F4041214
:1005510006EAD0E0FFD0E0FED0E0FDD0E0FC1205DD
:10056100B4D0E0F8E6FAEDD2E7CD33EC332482FBE8
:10057100E4C3CF33CFCE33CECD33CD33DBF37B07E3
:1005810075F00A846004F6081B0AE5F0F6088FF09E
:10059100740AA4FFACF08EF0740AA42CFEACF050E7
:1005A100010C8DF0740AA42CFDE435F0F608DBDEB5
:0305B100740722AA
:1005B400EC4D6011E8497017ED33EC3304600DE441
:1005C400FCFFFEFD22E933E8330470F802046D12E7
:1005D400043858046009E4CC2481500628500902E8
:1005E4000477284003020474C0E0EB4A7044B980E5
:1005F40006D0E0FB020463EF4E701CBD8008EBFFE5
:10060400EAFEE9FD80EBE98DF0A4FEE5F002069D2B
:10061400E9CDF9EAFEEBFFEF89F0A4FCE5F0CE8921
:10062400F0A42EFFE435F0CD89F0A42DFEE435F0DE
:100634008067EF4E7005BD80D780C3EF8BF0A4AC0C
:10064400F0EE8BF0A42CFCE435F0F8EF8AF0A42C47
:10065400E5F038FCE433CB8DF0A42CFCE5F03BF85A
:10066400EE8AF0A42CFCE5F038F8E433CF89F0A44A
:100674002CFCE5F038CF3400CE89F0A42FFFE5F050
:100684003EFEE433C98DF0A42EFEE5F039CD8AF0A8
:10069400A42FFFE5F03EFEE43DFD33D0E0FB500720
:1006A4000BBB000F020477EC2CFCEF33FFEE33FEA0
:0606B400ED33FD02044FCE
:1006BA003F8000004120000042C80000447A000048
:1006CA00461C400047C35000497424004B189680CA
:1006DA004CBEBC205A0E1BCA6753C21C749DC5AEC1
:1006EA00FB60065407601C2323120718EB5438607A
:1006FA00091207041207131205B4ECF8EDF9EEFA21
:10070A00EFCB22EB12071380F1543803241C900616
:10071A00BAFE93FC0EEE93FD0EEE930ECE93FF22DD
:03000000022209D0
:0C220900787FE4F6D8FD7581AA0222500F
:10072A00BB010689828A83E0225002E722BBFE02CD
:09073A00E32289828A83E4932200
:10074300BB010CE58229F582E5833AF583E022506B
:1007530006E92582F8E622BBFE06E92582F8E222B5
:0D076300E58229F582E5833AF583E49322CF
:10077000BB010689828A83F0225002F722BBFE0168
:02078000F32262
:10078200F8BB010DE58229F582E5833AF583E8F0AD
:10079200225006E92582C8F622BBFE05E92582C859
:0207A200F22241
:1007A400EF8DF0A4A8F0CF8CF0A428CE8DF0A42E69
:0207B400FE2223
:1007B600BC000BBE0029EF8DF084FFADF022E4CC27
:1007C600F875F008EF2FFFEE33FEEC33FCEE9DECF0
:1007D600984005FCEE9DFE0FD5F0E9E4CEFD22ED36
:1007E600F8F5F0EE8420D21CFEADF075F008EF2F80
:1007F600FFED33FD4007985006D5F0F222C398FD71
:050806000FD5F0EA220D
:0E080B00C3E49FFFE49EFEE49DFDE49CFC22FE
:10081900EB9FF5F0EA9E42F0E99D42F0E89C45F035
:0108290022AC
:0C082A00E0FCA3E0FDA3E0FEA3E0FF2241
:10083600A8828583F0D083D08212084D12084D120B
:10084600084D12084DE473E493A3C583C5F0C58330
:10085600C8C582C8F0A3C583C5F0C583C8C582C80C
:01086600226F
:10086700FAE6FB0808E6F925F0F618E6CA3AF62292
:10087700D083D082F8E4937012740193700DA3A310
:1008870093F8740193F5828883E473740293686024
:06089700EFA3A3A380DF24
:10089D00D083D082F8E4937012740193700DA3A3EA
:1008AD0093F8740193F5828883E473740293B5F021
:0D08BD00067403936860E9A3A3A3A380D889
:102D3D00EFB40A07740D122D48740A309811A89932
:102D4D00B8130CC2983098FDA899C298B811F630F6
:072D5D0099FDC299F59922CE
:1024F3008B438A448945E4F54BF54CE54A154AAECE
:1025030049700215494E6033AB46AA47A9481207E2
:102513002AFFAB43AA44A945054CE54CAC4B7002DA
:10252300054B14F5828C83EF120782EF60CD7401A3
:102533002548F548E43547F54780C0AB43AA44A98D
:0225430045222F
:102FDA00E4FFFE12072A600C0FEF70010E09E97078
:052FEA00F20A80EF2255
:1008CA00E709F608DFFA8046E709F208DFFA803E10
:1008DA0088828C83E709F0A3DFFA8032E309F608FD
:1008EA00DFFA806EE309F208DFFA806688828C8379
:1008FA00E309F0A3DFFA805A89828A83E0A3F60823
:10090A00DFFA804E89828A83E0A3F208DFFA804206
:10091A0080D280FA80C680D4805580F280298010E7
:10092A0080A680EA809A80A880DA80E280CA80293C
:10093A0088848C8589828A83E493A30586F0A3053B
:10094A0086DFF5DEF3800B89828A83E493A3F608B7
:10095A00DFF9ECFAA9F0EDFB2288848C8589828A7A
:10096A0083E0A30586F0A30586DFF6DEF480E3893B
:10097A00828A83E493A3F208DFF980D688F0EF60D5
:10098A00010E4E60CD88F0ED2402B4040050C3F588
:10099A0082EB2402B4040050B92323458223900930
:0209AA001A73BE
:1009AC00E709F60870FA8046E709F20870FA803E0B
:1009BC0088828C83E709F0A370FA8074E309F60847
:1009CC0070FA806CE309F20870FA806488828C8378
:1009DC00E309F0A370FA805889828A83E0A3F608B1
:1009EC0070FA804C89828A83E0A3F20870FA804006
:1009FC0080D280FA80C680D4805180F2802780100B
:100A0C0080A680EA809A80A880DA80E280CA80275B
:100A1C0088848C8589828A83E493A30586F0A30558
:100A2C008670F5800B89828A83E493A3F60870F9AB
:100A3C00ECFAA9F0EDFB2288848C8589828A83E00C
:100A4C00A30586F0A3058670F680E589828A83E487
:100A5C0093A3F20870F980D888F0ED2402B4040056
:100A6C0050CEF582EB2402B4040050C423234582FB
:050A7C00239009FC734A
:10221500021998E493A3F8E493A34003F68001F22E
:1022250008DFF48029E493A3F85407240CC8C333CA
:10223500C4540F4420C8834004F456800146F6DF99
:10224500E4800B0102040810204080903028E47ED1
:10225500019360BCA3FF543F30E509541FFEE4938E
:10226500A360010ECF54C025E060A840B8E493A355
:10227500FAE493A3F8E493A3C8C582C8CAC583CA80
:10228500F0A3C8C582C8CAC583CADFE9DEE780BE38
:013039000096
:00000001FF
